:100000009AEF25F00000000000EF00F00000000073
:100010000000000000000000F3D7FFFF0201DE51E6
:10002000000A32E0016A015007081CE303015DBFCA
:1000300002D0939E01D0938E060E0D6E0D2EFED72C
:100040000000938C060E0D6E0D2EFED70000939CC3
:10005000060E0D6E03010D2EFDD700005D375D917C
:10006000012AE1D7938E060E0D6E0D2EFED70000ED
:10007000938C060E0D6E0D2EFED70000939C060E7F
:100080000D6E0D2EFED7000012000201DE51000A97
:1000900018E0938C060E0D6E0D2EFED70000938E89
:1000A000060E0D6E0D2EFED70000939E060E0D6EF1
:1000B0000D2EFED70000939C060E0D6E0D2EFED762
:1000C00000001200086A096A100E0C6E013408362E
:1000D00009360450085E0550D8A0053C095ED8B02A
:1000E00007D0045008260550D8B0053C0926D89002
:1000F000003601360C2EEAD712000AAE029E000E20
:1001000012000201E551030159255C6FBEDFDEC21A
:100110005DF384DF03015D6B81DF03015851B00F94
:100120005D6F7CDF03015C510F0804E35CC35AF38D
:100130005B6B19D05CC302F00232029E0232029E57
:100140000232029E0232029E02C05BF302C000F045
:100150000036009000360090003600900036009087
:1001600000505C5D5A6F5AC35DF358DF03015B5169
:10017000100F5D6F53DF89DFDEC25DF34FDF400E8E
:1001800003015D6F4BDF12000201DE51000A12E035
:10019000939E060E0D6E0D2EFED70000938C060E5C
:1001A0000D6E0D2EFED70000938E060E0D6E0D2ED9
:1001B000FED7000012000B840BAEE6EF00F0010E3C
:1001C000036E026A016A006A0A360232FF0E1200EA
:1001D000220E0C6E086A096A0A6A0B6A0C06D8B409
:1001E0001FD0D8900B320A32093208320332023261
:1001F00001320032D8A0F2D70C06D8B409D004508E
:1002000008260550092206500A2207500B22EAD779
:10021000045008260550092206500A2207500B22D6
:100220001200026A016A006A086A036A000E12007C
:10023000A00E0301506F0F0E516F000E526F536FDF
:10024000A00E006E0F0E016E000E026E000E036E09
:100250004EC304F04FC305F0000E066E076EB8DF04
:1002600000C050F301C051F302C052F303C053F376
:10027000000E035C08E1000E025C05E1020E015C69
:1002800002E1940E005C01E231D0940E505F020E48
:10029000515B000E525B535B050E006E005007E091
:1002A0005333523351335033539FFF0FF8D750C35A
:1002B00000F051C301F052C302F053C303F0010E2A
:1002C000505F000E515B525B535B005001100210F7
:1002D00003100CE00000000000000000000000001F
:1002E00000000000000000000000E1D712000B80B9
:1002F0000BAE83EF01F0026A0AAEFF0E026E016ED2
:10030000006E0A360232FF0E12000301526B050E18
:10031000525D0AE252515025E16E000E5121E26E0B
:10032000200EE66E522BF3D752515025E16E000E8F
:100330005121E26EE66A520752515025536F000E6A
:100340005121546F0A0E046E000E056E4EC300F06C
:100350004FC301F0B7DE08C000F009C001F0300E55
:10036000002653C3E1FF54C3E2FF00C0E6FF0A0EBC
:10037000046E000E056E4EC300F04FC301F0A2DE06
:1003800000C04EF301C04FF3000E011802E1000E51
:10039000001801E102D05207CFD7120076DEDEC28C
:1003A0005DF33CDE400E03015D6F38DE4FC358F352
:1003B0004EC359F3A6DE0301536B5251535DD8B0BF
:1003C000B3D053515025E96E000E5121EA6EEE5024
:1003D000000A02E1556B09D053515025E96E000E19
:1003E0005121EA6E200EEE5C556F546B5451040897
:1003F000D8A092D0050E5503F3CF00F0F4CF01F052
:1004000054510026000E0122450E0024F66E500EB7
:100410000120F76E000EF86E000E01BEFF0EF822EE
:100420000900F5CF56F34F51020A000ED8A4010E71
:10043000016E4F51040A000ED8A4010E006E005048
:1004400001164F51060A000ED8A4010E006E01508D
:10045000001629E056B702D0579F01D0578F56B7E4
:1004600002D0579D01D0578D56B502D0579B01D071
:10047000578B56B502D0579901D0578956B302D041
:10048000579701D0578756B302D0579501D057855B
:1004900056B102D0579301D0578356B102D057912D
:1004A00001D0578120D056B502D0579F01D0578F29
:1004B00056B502D0579D01D0578D56B302D0579BE9
:1004C00001D0578B56B302D0579901D0578956B1F6
:1004D00002D0579701D0578756B102D0579501D017
:1004E00057855793579157C35DF398DD0201E65145
:1004F000040A010ED8A4000E016EE651050A010E91
:10050000D8A4000E006E0150001203E057C35DF343
:1005100085DD0301542B6AD75D6B80DD03015D6BC4
:100520007DDD0301532B49D74F51010F586F4EC347
:1005300059F3E7DD0301536B5251535DD8B0BBD083
:1005400053515025E96E000E5121EA6EEE50000A1B
:1005500002E1556B09D053515025E96E000E51212F
:10056000EA6E200EEE5C556F546B54510408D8A00F
:100570009AD0050E5503F3CF00F0F4CF01F054519B
:100580000026000E0122450E0024F66E500E0120BA
:10059000F76E000EF86E000E01BEFF0EF822090085
:1005A000F5CF56F34F51020A000ED8A4010E016E8A
:1005B0004F51040A000ED8A4010E006E005001161F
:1005C0004F51060A000ED8A4010E006E015000160D
:1005D00029E056BF02D0579F01D0578F56BF02D097
:1005E000579D01D0578D56BD02D0579B01D0578BD8
:1005F00056BD02D0579901D0578956BB02D05797A4
:1006000001D0578756BB02D0579501D0578556B9B0
:1006100002D0579301D0578356B902D0579101D0D9
:10062000578128D056BD02D0579F01D0578F56BD55
:1006300002D0579D01D0578D56BB02D0579B01D099
:10064000578B56BB02D0579901D0578956B902D063
:10065000579701D0578756B902D0579501D0578583
:1006600056B702D0579301D0578356B702D057914F
:1006700001D0578157C35DF3D1DC0201E651040A72
:10068000010ED8A4000E016EE651050A010ED8A491
:10069000000E006E0150001203E057C35DF3BEDC94
:1006A0000301542B62D75D6BB9DC03015D6BB6DCD3
:1006B0000301532B41D768DD12000B820BAE67EFAD
:1006C00003F003680268016800680A360232FF0E10
:1006D00012000C6A0E6A0250D8A482EF03F001C027
:1006E00002F000C001F0006A0E860250D8A482EF2A
:1006F00003F001C002F0016A0E960E880250D8B4D1
:1007000094EF03F00E50035ED8A4D8A099EF03F045
:10071000D89002BE9EEF03F0003601360236032E5B
:1007200089EF03F099EF03F0010E0C6E7ADDA1EF73
:1007300003F0020E0C6E3FDDA1EF03F0040E0C6E11
:10074000DCDC12001D0E0D6E0D2EFED71200030113
:100750004F6B0201E96B010EE86F4EC34FF30301CB
:100760004F374F914F374F914F374F914F374F91F1
:100770000201E75303E0080E03014F270201E8538B
:1007800003E0040E03014F270201E95303E0020EC8
:1007900003014F270201E05302E003014F2B75DCF8
:1007A000DEC25DF33BDC4FC35DF338DCEDDC060EEF
:1007B0000C6E300E0D6E0D2EFED70C2EFCD70000E9
:1007C000040E03014F5F61DCDEC25DF327DC4FC323
:1007D0005DF324DCD9DC060E0C6E300E0D6E0D2E92
:1007E000FED70C2EFCD7000012000B6A0A6A096AB9
:1007F00000500402F4CF09F0F3CF08F001500502D5
:10080000F4CF0BF0F3CF0AF000500502F3500926A5
:10081000F4500A22E86A0B2201500402F350092620
:10082000F4500A22E86A0B2208C000F009C001F067
:100830000AC002F00BC003F01200030144B102D061
:100840008A9201D08A8244B302D08A9401D08A84E9
:1008500044B502D0899401D0898444B702D08998E4
:1008600001D0898844B902D0899A01D0898A01C30C
:100870004EF302C34FF3DCDC12000CB07FEF04F048
:100880000CA227EF05F00E6A000E026496EF04F04A
:10089000F00E0214D8A461EF04F0023A01380F0BF5
:1008A00002260138F00B016E00380F0B01260038CC
:1008B000F00B006E08380F0B00260838F00B086E9E
:1008C0000E84D89002BE7AEF04F008360036013666
:1008D00002360E2A02BE7AEF04F0083600360136E0
:1008E00002360E2A02BE7AEF04F0083600360136D0
:1008F00002360E2A0E5003641BEF05F0035E0BBC9C
:1009000008AE21EF05F0D880800E08640030000E9C
:10091000002201220222D8A021EF05F0023201328A
:100920000032034A27EF05F021EF05F001C002F085
:1009300000C001F008C000F0086A000E0E860264D4
:10094000CDEF04F0F00E0214D8A4B5EF04F0023A93
:1009500001380F0B02260138F00B016E00380F0B27
:1009600001260038F00B006E0E84D89002BE7AEF9C
:1009700004F00036013602360E2A02BE7AEF04F089
:100980000036013602360E2A02BE7AEF04F0003637
:10099000013602360E2A7AEF04F001C002F000C0E0
:1009A00001F0006A000E0E960E880264FAEF04F061
:1009B000F00E0214D8A4E5EF04F0023A01380F0B50
:1009C00002260138F00B016E0E84D89002BE7AEF39
:1009D00004F0013602360E2A02BE7AEF04F0013628
:1009E00002360E2A02BE7AEF04F0013602360E2AD3
:1009F0007AEF04F001C002F0016A000E0E86026474
:100A00002CEF05F0F00E0214D8A409EF05F0023A1D
:100A10000E84D89002BE7AEF04F002360E2A02BE8F
:100A20007AEF04F002360E2A02BE7AEF04F00236A4
:100A30000E2A7AEF04F0010E0C6EDBEC00F030EFC2
:100A400005F0020E0C6E7DEC00F030EF05F0040EA8
:100A50000C6E33DE30EF05F0080E0C6E11EC01F079
:100A600012000450085E0550D8A0053C095E0650EF
:100A7000D8A0063C0A5E0750D8A0073C0B5E0336A0
:100A8000070E0C6E0334083609360A360B3604504E
:100A900003A00ED0085E0550D8A0053C095E0650A4
:100AA000D8A0063C0A5E0750D8A0073C0B5E0DD0CC
:100AB00008260550D8B0053C09260650D8B0063C9B
:100AC0000A260750D8B0073C0B2603360C2EDAD77F
:100AD0000234083609360A360B36045003A00ED00D
:100AE000085E0550D8A0053C095E0650D8A0063C1B
:100AF0000A5E0750D8A0073C0B5E0DD008260550B3
:100B0000D8B0053C09260650D8B0063C0A26075046
:100B1000D8B0073C0B260236070E0C6E023408369E
:100B200009360A360B36045002A00ED0085E055076
:100B3000D8A0053C095E0650D8A0063C0A5E0750C6
:100B4000D8A0073C0B5E0DD008260550D8B0053C58
:100B500009260650D8B0063C0A260750D8B0073CF4
:100B60000B2602360C2EDAD70134083609360A363F
:100B70000B36045002A00ED0085E0550D8A0053CEC
:100B8000095E0650D8A0063C0A5E0750D8A0073C74
:100B90000B5E0DD008260550D8B0053C092606503E
:100BA000D8B0063C0A260750D8B0073C0B260136C1
:100BB000070E0C6E0134083609360A360B3604501F
:100BC00001A00ED0085E0550D8A0053C095E065075
:100BD000D8A0063C0A5E0750D8A0073C0B5E0DD09B
:100BE00008260550D8B0053C09260650D8B0063C6A
:100BF0000A260750D8B0073C0B2601360C2EDAD750
:100C00000034083609360A360B36045001A00ED0DF
:100C1000085E0550D8A0053C095E0650D8A0063CE9
:100C20000A5E0750D8A0073C0B5E0DD00826055081
:100C3000D8B0053C09260650D8B0063C0A26075015
:100C4000D8B0073C0B260036070E0C6E0034083671
:100C500009360A360B36045000A00ED0085E055047
:100C6000D8A0053C095E0650D8A0063C0A5E075095
:100C7000D8A0073C0B5E0DD008260550D8B0053C27
:100C800009260650D8B0063C0A260750D8B0073CC3
:100C90000B2600360C2EDAD700B00ED004500826F2
:100CA0000550D8B0053C09260650D8B0063C0A26A7
:100CB0000750D8B0073C0B2612000B1E0A1E091E57
:100CC000081E082AD8B4092AD8B40A2AD8B40B2A8C
:100CD00012000B6A0B86FF0E1200830EC21644C36D
:100CE00000F000360090003600900050C2122ADD5D
:100CF000C282C2A201D0FDD7C4CF01F0006AC350A6
:100D00000012000E0112120003014A6B4B6B44C328
:100D10004CF345C34DF3800E4519006E800E005C08
:100D200002E1000E445D0BE2010E4A6F000E4B6FB4
:100D3000445100084C6F45C34DF3000E4D574CC352
:100D40004EF34DC34FF346C350F347C351F385EC05
:100D500001F0060E486F000E496F000E006E4951FB
:100D6000005C02E14851000819E248514625E16E55
:100D700049514721E26E010E485D006E000E49594F
:100D8000016E00504625E96E01504721EA6EEECF14
:100D9000E6FF010E485F000E495BDFD746C3E1FF67
:100DA00047C3E2FF200EE66E4A514B111AE0486B32
:100DB000496B48514625E96E49514721EA6EEE508C
:100DC000200A03E1484B492BF4D7010E485F000E7F
:100DD000495B48514625E16E49514721E26E2D0E8F
:100DE000E66E12000050086E0150006E016A026A41
:100DF000036A0B6A0C6A960E036E0A6A00C001F061
:100E000008C000F0086A026A64DC12000201E651C0
:100E1000040A010ED8A4000E016EE651050A010E67
:100E2000D8A4000E006E015000120DE045C34EF331
:100E300044C34FF346C350F347C351F348C352F37F
:100E4000CEEC01F059D0E651020A010ED8A4000EF2
:100E5000016EE651030A010ED8A4000E006E015087
:100E6000001214E0070E03014503F3CF4EF3040E06
:100E70004E2744C34FF34F374F9146C350F347C3F8
:100E800051F348C352F3CEEC01F036D0E06B44C3CB
:100E900000F000360090003600900050080F03016B
:100EA0004E6F55DC45C34EF352DC010EE06F03017B
:100EB000496B4851495D20E249514625E96E000ED3
:100EC0004721EA6EEECF01F001C04EF34E334E9F44
:100ED0004E334E9F4E334E9F4E334E9F38DC0301B0
:100EE00049514625E96E000E4721EA6EEECF4EF3DA
:100EF0002EDC0301492BDDD71200086A096A000EB7
:100F00000762036402EF08F0025006180A6E0750E9
:100F100003267E0ED8A093EF07F0035ED8B007EF4C
:100F200008F097EF07F0035ED8A00CEF08F0028EF0
:100F3000068E02C00EF001C00BF000C00DF0005094
:100F40000402F4CF0CF001500502F4CF00F0F3CF0F
:100F500008F00402F3500C26F4500822000E002280
:100F60000D500502F3500C26F4500822000E00220A
:100F700002500402F3500826F450002202500502E9
:100F8000016A000E0122F3500026F45001220D5098
:100F90000602F3500826F4500022026A000E0122D5
:100FA00002220B500602F3500026F4500122000EDC
:100FB00002220E500602F3500126F450022202BE15
:100FC000EAEF07F008360036013602360306D8B4D9
:100FD0000CEF08F0FDEF07F0D880800E08640030B9
:100FE000000E002201220222D8A0FDEF07F00232FB
:100FF00001320032034A07EF08F00AAE029E000EEB
:101000000FEF08F0010E11EC01F00FEF08F0020EE7
:101010005DEC03F00FEF08F0040EDBEC00F01200C3
:101020000B6A0350D8B456EF08F002500A6E028ED5
:101030008E0E035E03AE5AEF08F0036C080E035CDD
:10104000D8A035EF08F0036E013602C001F0026A45
:10105000080E035CD8A035EF08F0036E0136016A74
:101060000350D8A4D8903FEF08F00350D8B43FEF16
:1010700008F0D89002320132032E39EF08F00BBC91
:1010800001A04CEF08F0D8A04CEF08F0012AD8B42A
:10109000022A02BE69EF08F00AAE6FEF08F0021EE6
:1010A000011E012AD8B4022A6FEF08F0026A016A11
:1010B0006FEF08F00B800BAE73EF08F0026A0AAE18
:1010C00073EF08F0FF0E026E016E0A36023273EF04
:1010D00008F0010E0C6E77EC01F075EF08F0000ED1
:1010E0000C6E75EF08F0FF0E0C6E0150006E025092
:1010F000016E1200030144B102D08B9201D08B82A9
:1011000044B302D08B9401D08B8444B502D08B962B
:1011100001D08B8644B702D08B9801D08B8844B91C
:1011200002D08B9A01D08B8A01C34EF302C34FF3D6
:1011300018EC01F012000450000A12E10550000AF8
:101140000FE10650000A0CE10750000A09E1FF0E0A
:10115000006EFF0E016E7F0E026EFF0E036EA7D0B3
:10116000086A096A0750D8B446EF09F00350D8B4AA
:101170004AEF09F0025006180A6E028E068E0E6AB9
:1011800002C008F001C00CF000C00DF004500D5E6C
:101190000550D8A0053C0C5E0650D8A0063C085E61
:1011A000086A0C6A0D6AD8A0DDEF08F0D890023208
:1011B000013200320832010E0E6E0750035ED8A0D5
:1011C000EAEF08F07E0E0E240326D8B04FEF09F0A8
:1011D000F0EF08F07E0E0E240326D8A054EF09F09D
:1011E000180E0B6E0D360C360836003601360236F8
:1011F0000E360450005E0550D8A0053C015E065036
:10120000D8A0063C025E06340E120EA00BEF09F0C9
:101210000D8016EF09F0045000260550D8B0053CAB
:1012200001260650D8B0062802260D900B2EF2EFAC
:1012300008F03CEF09F0D8900036013602360E3641
:101240000450005E0550D8A0053C015E0650D8A0B1
:10125000063C025E06340E10010B0D26D8B00C2A97
:10126000D8B4082AD8A43CEF09F008320C320D3269
:10127000032AD8B44FEF09F00AAE089E0850026E58
:101280000C50016E0D50006E57EF09F0010E21DD7C
:1012900057EF09F0020E11EC01F057EF09F0040EC0
:1012A0005DEC03F057EF09F0080EDBEC00F01200E4
:1012B000025006180E6E086A096A0B6A035007642A
:1012C0004BEF0AF006500A6E068E028E03500B6E2C
:1012D0000750036E000E0B649BEF09F00B50075E86
:1012E000D8B43CEF0AF0070E07640AEF0AF0075E75
:1012F00000C008F001C000F002C001F0026A074E11
:101300003CEF0AF00764DFEF09F0075E00C008F069
:1013100001C000F0016A074E3CEF0AF00764BDEF20
:1013200009F0075E00C008F0006A074E3CEF0AF0C3
:101330000764A4EF09F00AC002F005C001F004C080
:1013400000F0086A68EF0BF0030E0764AFEF09F0D6
:10135000075E08380F0B086E074E3CEF0AF0D89076
:101360000832074E3CEF0AF0D8900832074E3CEFA7
:101370000AF0D89008323CEF0AF0030E0764CEEF73
:1013800009F0075E08380F0B086E0038F00B0826CE
:1013900000380F0B006E074E3CEF0AF0D890003279
:1013A0000832074E3CEF0AF0D89000320832074E60
:1013B0003CEF0AF0D890003208323CEF0AF0030EFE
:1013C0000764F6EF09F0075E08380F0B086E003867
:1013D000F00B082600380F0B006E0138F00B0026CA
:1013E00001380F0B016E074E3CEF0AF0D890013226
:1013F00000320832074E3CEF0AF0D890013200323A
:101400000832074E3CEF0AF0D89001320032083221
:101410003CEF0AF0030E076427EF0AF0075E083876
:101420000F0B086E0038F00B082600380F0B006E0B
:101430000138F00B002601380F0B016E0238F00B5B
:10144000012602380F0B026E074E3CEF0AF0D890CF
:101450000232013200320832074E3CEF0AF0D890D7
:101460000232013200320832074E3CEF0AF0D890C7
:101470000232013200320832096A000E0EAE30EF3D
:101480000BF0081E001E011E021E082A0022012267
:10149000022230EF0BF00750D8A451EF0AF068EFAA
:1014A0000BF0096A02C00AF0028E068E0750035C38
:1014B000076ED8B423EF0BF0070E0764F1EF0AF0C4
:1014C000075E0450096E0550046E0650056E066AEC
:1014D000074E23EF0BF0070E0764C6EF0AF0075E16
:1014E0000450096E0550046E056A074E23EF0BF099
:1014F000070E0764A4EF0AF0075E0450096E046A41
:10150000074E23EF0BF0070E07648BEF0AF00AC0BB
:1015100002F068EF0BF0030E076496EF0AF0075E27
:1015200009380F0B096E074E23EF0BF0D8900932E4
:10153000074E23EF0BF0D8900932074E23EF0BF044
:10154000D890093223EF0BF0030E0764B5EF0AF0D1
:10155000075E09380F0B096E0438F00B09260438B2
:101560000F0B046E074E23EF0BF0D89004320932B4
:10157000074E23EF0BF0D89004320932074E23EFC9
:101580000BF0D8900432093223EF0BF0030E0764FE
:10159000DDEF0AF0075E09380F0B096E0438F00B17
:1015A000092604380F0B046E0538F00B04260538A5
:1015B0000F0B056E074E23EF0BF0D8900532043267
:1015C0000932074E23EF0BF0D8900532043209326E
:1015D000074E23EF0BF0D89005320432093223EF87
:1015E0000BF0030E07640EEF0BF0075E09380F0BCC
:1015F000096E0438F00B092604380F0B046E053809
:10160000F00B042605380F0B056E0638F00B052687
:1016100006380F0B066E074E23EF0BF0D8900632FC
:10162000053204320932074E23EF0BF0D890063210
:10163000053204320932074E23EF0BF0D890063200
:10164000053204320932086A000E0EAE30EF0BF09C
:10165000091E041E051E061E092A04220522062252
:10166000095008260450002205500122065002228B
:101670000EBE47EF0BF0D8A056EF0BF0023201324E
:1016800000320832033E56EF0BF062EF0BF0D8B099
:101690005CEF0BF0000E081E001E011E021E082A41
:1016A0000022012202220A7E5CEF0BF0010E0C6E7A
:1016B0003DEC04F06AEF0BF0020E0C6E3DEC04F012
:1016C0006AEF0BF0040E0C6E5DEC03F06AEF0BF0AA
:1016D000000E0C6E12000201DB6B5F6B0301446BAA
:1016E0001DEC04F05FC244F305DD01C34EF302C3F9
:1016F0004FF318EC01F0120004000201DB51DC1979
:10170000000ED8A4010E016EDA51DD19000ED8A426
:10171000010E006E01500012D8B425D1DBC2DCF2FC
:1017200003011D6B1E6B0201DBA105D003010D51EE
:101730001D270E511E230201DBA305D003010B510F
:101740001D270C511E230201DBA505D003011151F9
:101750001D2712511E230201DBA705D003010F51E3
:101760001D2710511E230201DBA905D003010951D9
:101770001D270A511E2303010051000A000ED8A4A0
:10178000010E016E0051010A000ED8A4010E006E78
:1017900001500016D8B488D01DC344F31EC345F3CE
:1017A000F70E466F020E476F84EC06F00201F95106
:1017B000200A03E0F9C2F0F202D0300EF06F2E0ED4
:1017C000F16FFA51200A03E0FAC2F2F202D0300EB1
:1017D000F26FFB51200A03E0FBC2F3F202D0300E9D
:1017E000F36F03010051040A010ED8A4000E016E2C
:1017F0000051050A010ED8A4000E006E015000121F
:101800002AE00201DA51010A04E1040E0301426FE9
:1018100003D00301060E426F0201DA51DD190DE01B
:1018200042C344F3100E0301456FAD0E466F020E26
:10183000476F080E486F06EC07F042C344F3280ECA
:101840000301456FF00E466F020E476F040E486F9E
:1018500006EC07F028D00201DA51010A03E1030186
:10186000426B03D00301010E426F0201DA51DD1910
:101870000DE042C344F3090E0301456FBE0E466FEF
:10188000020E476F080E486F06EC07F042C344F3A0
:101890000B0E0301456FF00E466F020E476F040EEC
:1018A000486F06EC07F05FD003010051000A5BE0CF
:1018B0000DC300F00EC301F001320032019E01BCE5
:1018C000018E01AE03D002E3004A012A03011D513B
:1018D00000261E51012200C01DF301C01EF300C0EE
:1018E00044F301C045F3F70E466F020E476F84ECD8
:1018F00006F00201F951200A03E0F9C2F0F202D029
:10190000300EF06F2E0EF16FFA51200A03E0FAC28A
:10191000F2F202D0300EF26FDA51010A03E1030154
:10192000426B03D00301010E426F0201DA51DD194F
:101930000DE042C344F3090E0301456FB60E466F36
:10194000020E476F070E486F06EC07F042C344F3E0
:101950000B0E0301456FF00E466F020E476F030E2C
:10196000486F06EC07F002015F51D919000ED8A4A8
:10197000010E016EDA51DD19000ED8A4010E006EC1
:1019800001500012D8B4EBD05FC2D9F203011D6B35
:101990001E6B02015FA105D0030117511D271851CD
:1019A0001E2302015FA305D003011B511D271C51FB
:1019B0001E2302015FA505D0030119511D271A51ED
:1019C0001E2302015FA705D0030115511D271651E3
:1019D0001E2302015FA905D0030113511D271451D5
:1019E0001E2303010051000A000ED8A4010E016E4F
:1019F0000051010A000ED8A4010E006E015000161D
:101A0000D8B474D01DC344F31EC345F3F70E466F1C
:101A1000020E476F84EC06F0F9C2F0F2FAC2F1F25E
:101A2000FBC2F2F2FCC2F3F20051040A010ED8A488
:101A3000000E016E0051050A010ED8A4000E006EC2
:101A4000015000122AE00201DA51010A04E1060EF7
:101A50000301426F03D00301040E426F0201DA5109
:101A6000DD190DE042C344F3100E0301456FD00EA3
:101A7000466F020E476F080E486F06EC07F042C330
:101A800044F3280E0301456FF00E466F020E476FB8
:101A9000040E486F06EC07F028D00201DA51010A63
:101AA00004E1010E0301426F02D00301426B020107
:101AB000DA51DD190DE042C344F3090E0301456F0D
:101AC000C70E466F020E476F080E486F06EC07F010
:101AD00042C344F30B0E0301456FF00E466F020E36
:101AE000476F040E486F06EC07F039D01DC344F36E
:101AF0001EC345F3F70E0301466F020E476F84ECD9
:101B000006F0FAC2F0F2FBC2F1F2FCC2F2F20201FC
:101B1000DA51010A04E1010E0301426F02D0030110
:101B2000426B0201DA51DD190DE042C344F3090EA4
:101B30000301456FFC0E466F010E476F070E486F9D
:101B400006EC07F042C344F30B0E0301456FF00EA1
:101B5000466F020E476F030E486F06EC07F0040055
:101B6000DAC2DDF20201AC51000AD8A489D0030127
:101B70000051040A010ED8A4000E016E0051050A9E
:101B8000010ED8A4000E006E015000123BE00001CF
:101B9000F753010ED8A4000E006E02019D510016ED
:101BA0000DE00301446B700E456FF50E466F000E9D
:101BB000476F010E486F06EC07F023D002019D53DA
:101BC000010ED8A4000E006E0001F75100160DE0C2
:101BD0000301446B700E456FF30E466F000E476FA6
:101BE000010E486F06EC07F00CD00301446B700E39
:101BF000456FFC0E466F000E476F010E486F06ECF6
:101C000007F03ED003010051000A3AE00001F7530B
:101C1000010ED8A4000E006E02019D5100160DE0C9
:101C20000301446B080E456FFA0E466F000E476FB6
:101C3000010E486F06EC07F023D002019D53010E00
:101C4000D8A4000E006E0001F75100160DE003014C
:101C5000446B080E456FF80E466F000E476F010E7D
:101C6000486F06EC07F00CD00301446B080E456F7B
:101C7000F10E466F000E476F010E486F06EC07F03D
:101C800004001200A6A202D00000FCD7A69C42C30A
:101C9000A9FF43C3A8FFA69EA684F2CF00F0F29E40
:101CA000550EA76EAA0EA76EA68200BE02D0F29EA7
:101CB00001D0F28EA694A1B802D00000FCD7A19862
:101CC0001200030E0C6E950E0D6E0D2EFED70C2E0F
:101CD000FCD712000301446B6DEC06F0F2EC06F049
:101CE000890E046E410E056E1C0E066E810E076E87
:101CF0007DEC07F010EC08F01200010E0301446FB8
:101D00006DEC06F0F2EC06F0890E046E410E056EE5
:101D10001C0E066E810E076E7DEC07F010EC08F0CD
:101D2000120000C008F00150006E016A026A036AE6
:101D30000B6A0C6A016A026A036A960E036E0A6AEB
:101D400000AEA9EF0EF0081E001E082AD8B4002A23
:101D50000A8E00C001F008C000F0086A026A69EC4F
:101D600003F012000450000A12E10550000A0FE1CE
:101D70000650000A0CE10750000A09E1FF0E006E50
:101D8000FF0E016EFF0E026E7F0E036E99D00C6A7D
:101D900007BE0C2A0D6A0B6A0A6A096A086A0350B0
:101DA000021001100010D8B485D0035007180E6E31
:101DB0000EBE0D1E07AE0BD0041E051E061E071E0E
:101DC000042AD8B4052AD8B4062AD8B4072A03AE00
:101DD0000BD0001E011E021E031E002AD8B4012AC9
:101DE000D8B4022AD8B4032A035007100E6E0EBED0
:101DF0001DD031EC05F00CBE36D00DAE5BD0001E10
:101E0000011E021E031E002AD8B4012AD8B4022AD9
:101E1000D8B4032A081E091E0A1E0B1E082AD8B4AD
:101E2000092AD8B40A2AD8B40B2A44D007AE15D050
:101E300003BE0DD003500B6E02500A6E0150096EA6
:101E40000050086E036A026A016A006AD6D7036A04
:101E5000026A016A006A002A000C031E021E011EAB
:101E6000001E0C8EC6D7082AD8B4092AD8B40A2A6C
:101E7000D8B40B2A0450085CD8A4BFD70550095C1D
:101E8000D8A4BBD706500A5CD8A4B7D707500B5CC0
:101E9000D8A4B3D70B6A0A6A096A086A002AD8B4B8
:101EA000012AD8B4022AD8B4032A03AEA6D70E6AF0
:101EB0000E88FF0C0E6A0CA002D05DEC06F0000F3D
:101EC000120042C300F043C301F0030E046E000E83
:101ED000056EF5EC03F000C042F301C043F3800E41
:101EE000026E800E0118025C02E10050500803E30C
:101EF000006A016ABCD0800E006E800E0301431997
:101F0000005C02E14251AB0805E3F40E4227000EEB
:101F10004323A9D0800E010A006E800E4319005C95
:101F200002E14251480805E3FE0E4227000E43231A
:101F30009AD0800E020A006E800E4319005C02E106
:101F40004251460805E3180E4227010E43238BD069
:101F5000800E030A006E800E4319005C02E14251BC
:101F6000340805E3290E4227010E43237CD0800E5E
:101F7000040A006E800E4319005C02E142514C08D5
:101F800005E3360E4227010E43236DD0800E080A6A
:101F9000006E800E4319005C02E14251850805E3A2
:101FA000AE0E4227010E43235ED0800E0C0A006E57
:101FB000800E4319005C02E14251FA0805E3E40E89
:101FC0004227010E43234FD0800E120A006E800E6E
:101FD0004319005C02E142510F0805E3120E42274B
:101FE000020E432340D0800E160A006E800E431965
:101FF000005C02E14251E60805E3880E4227020E2A
:10200000432331D0800E1B0A006E800E4319005C02
:1020100002E14251EA0805E3E70E4227020E43239C
:1020200022D0800E210A006E800E4319005C02E16E
:102030004251360805E3340E4227030E432313D0E2
:10204000800E290A006E800E4319005C02E14251A5
:10205000040805E3840E4227030E432304D0520EE6
:102060004227030E432342C300F043C301F0120092
:10207000040030DE00C036F301C037F3000E01BEAD
:10208000FF0E0301386F396F38DE00C03AF301C02C
:102090003BF3000E01BEFF0E03013C6F3D6F36C3E4
:1020A00042F337C343F30DDF3CDE00C03EF301C013
:1020B0003FF302C040F303C041F3800E03013D191A
:1020C000006E800E3919005C08E138513C5D05E175
:1020D00037513B5D02E136513A5D08E3E70E366F5A
:1020E000030E376F000E386F396F44D03A513625E2
:1020F000006E3B513721016E3C513821026E3D513B
:102100003921036E640E046E000E056E066E076EB6
:10211000E8EC00F036C304F037C305F038C306F02E
:1021200039C307F03A51045E3B51055A3C51065AF7
:102130003D51075A17DE00C036F301C037F302C025
:1021400038F303C039F3800E046E800E0318045C6C
:1021500008E10250000805E10150030802E10050C7
:10216000E70808E2E70E0301366F030E376F000E33
:10217000386F396F3EC300F03FC301F040C302F037
:1021800041C303F0000E046E000E056E200E066EB5
:10219000820E076E7DEC07F0000E046E000E056ED9
:1021A0007A0E066E880E076E9BEC08F000C03EF3B8
:1021B00001C03FF302C040F303C041F3F40E046ECC
:1021C000FD0E056E340E066E7F0E076E9BEC08F05A
:1021D00000C03EF301C03FF302C040F303C041F32F
:1021E00000C004F001C005F002C006F003C007F013
:1021F0007DEC07F0000E046E000E056E200E066EDC
:10220000810E076E9BEC08F000C03EF301C03FF367
:1022100002C040F303C041F3000E046E000E056ED1
:10222000000E066E7E0E076E58EC09F000C03EF3FD
:1022300001C03FF302C040F303C041F310EC08F0CB
:1022400000C003F301C004F3800E0118026E800E7B
:10225000025C02E10A0E005C06E2010E0301076F58
:10226000000E086F19D00301800E3919006E800E20
:10227000005C08E1000E385D05E1000E375D02E10B
:10228000640E365D05E2E70E076F030E086F04D09B
:1022900036C307F337C308F3120001340836093692
:1022A0000450085E0550D8A0053C095E0036013692
:1022B0000F0E0C6E013408360936045000A006D00B
:1022C000085E0550D8A0053C095E05D008260550DB
:1022D000D8B0053C0926003601360C2EEBD700B0ED
:1022E00006D0045008260550D8B0053C0926000049
:1022F000120003013C6B38C301F0010E006E015067
:1023000004E000360090FF0FFBD700C03BF336C35C
:10231000E9FF37C3EAFF0050EE14016E0152010ECF
:10232000D8A4000E006E3A51001A18E03951000886
:1023300004E2C7DCC6DC3907F9D736C3E9FF37C387
:10234000EAFF3B51EE14016E0152010ED8A4000EBB
:10235000006E3A51001A02E0FF0E3C6F3CC300F0E1
:1023600012006BEC0BF0FF0E426F436B8BDCFE0E2A
:102370000301426F436B86DCFD0E0301426F436B2A
:1023800081DC7CEC0BF003010051000A02E18A8C35
:102390008A8E899E89868B908B9C8B9E076B086B9F
:1023A000036B046B02019B6B9C6B03010051040ADD
:1023B000010ED8A4000E016E0051050A010ED8A42A
:1023C000000E006E0150001236E0020E446F100E37
:1023D000456F100E466F010E476F080E486F06ECF2
:1023E00007F004000D0E0B6E2D0E0C6ED70E0D6E49
:1023F0000D2EFED70C2EFCD70B2EFAD700000000B6
:10240000020E0301446F100E456F070E466F010E5A
:10241000476F080E486F06EC07F00301446B100E7F
:10242000456FFE0E466F000E476F080E486F06ECB4
:1024300007F0040036D003010051000A32E0010E1B
:10244000446F456B2B0E466F010E476F080E486FA9
:1024500006EC07F004000D0E0B6E2D0E0C6ED70E61
:102460000D6E0D2EFED70C2EFCD70B2EFAD70000CA
:102470000000010E0301446F456B220E466F010EF2
:10248000476F080E486F06EC07F00301446B456B7D
:10249000190E466F010E476F080E486F06EC07F0E5
:1024A00004001200E5DD800E0419026E800E0201A8
:1024B000EF19025C03E1EE510301035D010ED8B098
:1024C000000E026E800E0201ED19016E800E0301F6
:1024D0000419015C03E103510201EC5D0201010EEC
:1024E000D8B0000E016E800E006E800EED19005CFB
:1024F00002E1EC510008010ED8B0000E006E015050
:102500000016025000122DE00400B2DD810E366F7D
:102510000F0E376F386B050E396F010E3A6FE9DE1B
:10252000005203E0010E02015E6F02015E51010ADA
:10253000010ED8A4000E0301356F810E366F0F0E09
:10254000376F386B050E396F3A6BD3DE3551001695
:1025500007E007DF0301076B086B006A016A05D01B
:10256000A2D707C300F008C301F012000450000A0C
:1025700008E10550000A05E1FF0E006E7F0E016EB6
:1025800057D00D6A096A086A01500010D8B4000CCF
:10259000015005180A6E0ABE0D1E0B6A05AE05D065
:1025A000041E051E042AD8B4052A01AE05D0001E5B
:1025B000011E002AD8B4012A015005100A6E0ABE75
:1025C00010D06BDE0BB020D00DAE000C001E011E33
:1025D000002AD8B4012A081E091E082AD8B4092ADC
:1025E000000C05AE0DD001BE07D00150096E0050A1
:1025F000086E016A006AE8D7016A006A002A000CC6
:10260000011E001E0B2ADDD7082AD8B4092A04505F
:10261000085CD8A4D9D70550095CD8A4D5D7096AD5
:10262000086A002AD8B4012A01AECED70000FF0CF8
:102630001200030E0301326F02015F6B0301446B52
:102640007AEC08F02FDF00C033F301C034F333C35A
:1026500007F334C308F3140E046E000E056E33C383
:1026600000F034C301F082DF005003013325306FE6
:1026700001503421316F32C32FF32F511F0847E32C
:102680002FC344F37AEC08F00DDF00C007F301C05C
:1026900008F3800E0118026E800E03013119025CEE
:1026A00002E13051005C31E2140E046E000E056E42
:1026B00007C300F008C301F059DF005003010725EC
:1026C000306F01500821316F2FC35FF232C360F2C7
:1026D000800E0819006E800E005C02E1780E075D26
:1026E00001E215D032512F25016E01C02FF30150A8
:1026F000090A03E1080E2F6F07D02F51110A04E1D8
:10270000100E2F6F040E326F01D001D0B6D75FC20A
:1027100044F37AEC08F0120060C229F30201605120
:102720005F25016E01C02BF301501F0803E21F0E4D
:1027300003012B6F02015F510301295D06E229515C
:1027400002015F5D03012C6F01D02C6B2CC35FF283
:102750002CC344F37AEC08F0A5DE00C007F301C0F7
:1027600008F3000E011802E1000E001801E173D019
:1027700007C32DF308C32EF303012C51010F2A6F59
:102780002A512B5DD8A063D02AC344F37AEC08F019
:1027900089DE00C007F301C008F3000E011802E152
:1027A000000E001801E157D0800E03010819006ED9
:1027B000800E2E19005C02E12D51075D0FE3340EEF
:1027C0000C6EF10E0D6E0D2EFED70C2EFCD70000F8
:1027D000000068DE00C007F301C008F3800E0301AB
:1027E0000819006E800E2E19005C02E12D51075D64
:1027F0000FE3340E0C6EF10E0D6E0D2EFED70C2E67
:10280000FCD7000000004EDE00C007F301C008F353
:10281000800E03010819006E800E2E19005C02E183
:102820002D51075D11E207C32DF308C32EF32AC310
:102830005FF2800E0819006E800E005C02E1780ED7
:10284000075D01E204D001D002D02A2B99D75FC2E4
:1028500044F37AEC08F01200030129B102D0899CFC
:1028600001D0898C01C34EF302C34FF318EC01F081
:102870001200030E03012E6F2A6B2EC334F1030ED8
:102880002B6F140E046E000E056E07C300F008C314
:1028900001F06CDE0050030107252C6F0150082168
:1028A0002D6F2EC329F329511F084CE329C344F38C
:1028B0001DEC04F0BEDEF6DD00C007F301C008F336
:1028C000800E0118026E800E03012D19025C02E1D8
:1028D0002C51005C35E2140E046E000E056E07C329
:1028E00000F008C301F042DE0050030107252C6F01
:1028F000015008212D6F29C3DBF25FC22AF32EC3DA
:1029000034F160C22BF3800E0819006E800E005C5B
:1029100002E1780E075D01E215D02E512925016EE6
:1029200001C029F30150090A03E1080E296F07D0FD
:102930002951110A04E1100E296F040E2E6F01D0E7
:1029400001D0B1D72AC35FF2DBC244F31DEC04F01F
:102950005FC244F37AEC08F02BC360F2340E0C6EC5
:10296000F10E0D6E0D2EFED70C2EFCD700000000D0
:10297000120034C129F3010134510201DB25016E3B
:1029800001C02BF301501F0803E21F0E03012B6F40
:102990000201DB510301295D06E229510201DB5DE1
:1029A00003012C6F01D02C6B2CC3DBF22CC344F33E
:1029B0001DEC04F077DD00C007F301C008F3000E42
:1029C000011802E1000E001801E173D007C32DF3D6
:1029D00008C32EF303012C51010F2A6F2A512B5DDE
:1029E000D8A063D02AC344F31DEC04F05BDD00C023
:1029F00007F301C008F3000E011802E1000E0018F1
:102A000001E157D0800E03010819006E800E2E19C7
:102A1000005C02E12D51075D0FE3340E0C6EF10EE8
:102A20000D6E0D2EFED70C2EFCD7000000003ADDF7
:102A300000C007F301C008F3800E03010819006EFF
:102A4000800E2E19005C02E12D51075D0FE3340E5C
:102A50000C6EF10E0D6E0D2EFED70C2EFCD7000065
:102A6000000020DD00C007F301C008F3800E030161
:102A70000819006E800E2E19005C02E12D51075DD1
:102A800011E207C32DF308C32EF32AC3DBF2800E35
:102A90000819006E800E005C02E1780E075D01E20D
:102AA00004D001D002D02A2B99D7DBC244F31DEC0D
:102AB00004F01200810E0301366F0F0E376F386B72
:102AC000320E396F3A6B15DC00C029F3810E366F78
:102AD0000F0E376F040E386F320E396F3A6B09DC08
:102AE00000502913810E366F0F0E376F050E386FA9
:102AF000320E396F3A6B79EC11F02951001203E074
:102B0000010E0201906F1200040003012A5102011C
:102B10008F1903E18E5103012919D8B480D0030124
:102B200029C38EF22AC38FF2000E2A1902E1010E88
:102B3000291930E10051040A010ED8A4000E016EDB
:102B40000051050A010ED8A4000E006E01500012BB
:102B50000DE0020E446F400E456F960E466F020E5A
:102B6000476F040E486F06EC07F010D003010051C8
:102B7000000A0CE0010E446F040E456F910E466F83
:102B8000020E476F040E486F06EC07F002018E6BD1
:102B90008F6B45D029C38EF22AC38FF229C344F329
:102BA0002AC345F3F70E0301466F020E476F84EC0C
:102BB00006F0FAC2F0F22E0E0201F16FFBC2F2F241
:102BC000FCC2F3F203010051040A010ED8A4000E66
:102BD000016E0051050A010ED8A4000E006E0150CE
:102BE00000120DE0020E446F400E456FF00E466F6E
:102BF000020E476F040E486F06EC07F010D0030179
:102C00000051000A0CE0010E446F040E456FF00EF7
:102C1000466F020E476F040E486F06EC07F0040083
:102C20001200040002015E6B3DDC800E03010819F6
:102C3000006E800E005C02E16E0E075D01E258D16D
:102C40006BEC0BF0020E0B6E040E0C6EBA0E0D6EDA
:102C50000D2EFED70C2EFCD70B2EFAD7000022DC4F
:102C6000800E03010819006E800E005C02E16E0EFA
:102C7000075D01E23DD1800E016E800E0201EB196D
:102C8000015C02E1EA516E08010ED8B0000E016E3F
:102C9000800EEB19006E800E03010819005C03E141
:102CA00007510201EA5D010ED8B0000E006E01501E
:102CB000001601E01DD107C323F308C324F3D9DDB7
:102CC000000E081902E1000E071903E16BEC0BF08E
:102CD0000FD152EC12F0800E03010819006E800E25
:102CE000005C02E1780E075D01E202D142DE000ED7
:102CF0000301081902E1000E071903E16BEC0BF068
:102D0000F7D052EC12F0800E03010819006E800E0D
:102D1000005C02E1780E075D01E2EAD0FDDC000E06
:102D20000301081902E1000E071903E16BEC0BF037
:102D3000DFD052EC12F0800E03010819006E800EF5
:102D4000005C02E1780E075D01E2D2D0800E081926
:102D5000016E800E015C02E1C80E075D010ED8B065
:102D6000000E016E800E0819006E800E2419005CA2
:102D700002E12351075D010ED8B0000E006E005035
:102D80000114036E0751235D016E08512459026E30
:102D9000800E006E800E0218005C02E10150640893
:102DA000010ED8B0000E006E0350001601E0A0D056
:102DB00007C323F308C324F3DBC225F3000E266FF9
:102DC0005FC227F3000E286F0201DA51010A02E107
:102DD000DA6B02D0010EDA6F6BEC0BF0DAC229F37A
:102DE0003BDD020E0B6E040E0C6EBA0E0D6E0D2E38
:102DF000FED70C2EFCD70B2EFAD7000052EC12F0A7
:102E0000800E03010819006E800E005C02E1780E4E
:102E1000075D01E26DD02DDD000E081902E1000E04
:102E2000071903E16BEC0BF063D052EC12F0800E4B
:102E300003010819006E800E005C02E1780E075D48
:102E400001E256D096DD000E0301081902E1000EE2
:102E5000071903E16BEC0BF04BD052EC12F0800E33
:102E600003010819006E800E005C02E1780E075D18
:102E700001E23ED051DC000E0301081902E1000E10
:102E8000071903E16BEC0BF033D052EC12F0800E1B
:102E900003010819006E800E005C02E1780E075DE8
:102EA00001E226D0800E2419006E800E0819005C05
:102EB00002E10751235D1BE20201DA51010A02E13E
:102EC000DA6B02D0010EDA6FDAC229F3C5DC25C352
:102ED000DBF227C35FF225C344F31DEC04F05FC2AD
:102EE00044F37AEC08F023C307F324C308F3040087
:102EF000120045EC00F0DEC25DF30EEC00F0800E37
:102F000003015D6F0EEC00F023C35DF30EEC00F0E7
:102F1000C4EC00F012000301276B286B640E020161
:102F2000FE5D0301246F000E0201FF590301256FAE
:102F3000036B046B010E0201AA6F000EAB6F04005D
:102F4000AC5304E0280E0301266F03D00301780E72
:102F5000266F236B2651235D4EE20201AC51000A1D
:102F6000010ED8A4000E016E81B002D0068001D0FF
:102F7000069081B802D0D88001D0D89006B003D096
:102F800002E2069001D0068081BA02D0D88001D03A
:102F9000D89006B003D002E2069001D00680006A05
:102FA00006B0002A0150001607E084DD02019051AE
:102FB000010A02E1906B35D338EC10F0800E28192D
:102FC000006E800E0419005C02E10351275D08E2E7
:102FD00003C327F304C328F307C3AAF208C3ABF261
:102FE000100E0C6E940E0D6E0D2EFED70C2EFCD70F
:102FF0000000232BAFD7040027C305F328C306F333
:10300000AAC229F3ABC22AF37FDD800E0201AB19FD
:10301000006E800EFF19005C02E1FE51AA5D000EF9
:10302000D8B0010E006E00509D15056E800E9C19E3
:10303000036E800EAB19035C02E1AA519B5D010E89
:10304000D8B0000E036E9B51AA5D016E9C51AB5926
:10305000026E800E03012519006E800E0218005CBE
:1030600002E10150245D010ED8B0000E006E005048
:103070000314046E800E0201AB19036E800E9C19BE
:10308000035C02E19B51AA5D010ED8B0000E036EF5
:10309000AA519B5D016EAB519C59026E800E0301DB
:1030A0002519006E800E0218005C02E10150245DBB
:1030B000010ED8B0000E006E035000160050041030
:1030C000016E02019C51030A02E1E70E9B19010EF9
:1030D000D8A4000E006E015000120550001602E048
:1030E000010E9E6FAC51000A010ED8A4000E016EB5
:1030F00081B002D0068001D0069081B202D0D88083
:1031000001D0D89006B003D002E2069001D006802C
:1031100081B402D0D88001D0D89006B003D002E2AA
:10312000069001D00680006A06B0002A0150001601
:1031300007E0C0DC02019051010A02E1906B71D2FC
:10314000030106510201A91903E1A8510301051960
:10315000D8B477D0030105C3A8F206C3A9F2800E44
:103160000619006E800E005C02E1640E055D1EE330
:10317000050E0525006E000E0621016E00C005F348
:1031800001C006F300C044F301C045F3F70E466FDB
:10319000020E476F84EC06F0F9C2F0F2FAC2F1F2C7
:1031A000FBC2F2F2570E0201F36F20D005C344F3C5
:1031B00006C345F3F70E0301466F020E476F84EC1A
:1031C00006F00201FB51200A03E0FBC2F0F202D03C
:1031D000300EF06F2E0EF16FFC51200A03E0FCC29E
:1031E000F2F202D0300EF26F570EF36F030100516E
:1031F000040A010ED8A4000E016E0051050A010E4A
:10320000D8A4000E006E015000120CE0446B400E7A
:10321000456FF00E466F020E476F040E486F06ECC6
:1032200007F00FD003010051000A0BE0446B040EBD
:10323000456FF00E466F020E476F040E486F06ECA6
:1032400007F00201AC51000A010ED8A4000E016E75
:1032500081B002D0068001D0069081B202D0D88021
:1032600001D0D89006B003D002E2069001D00680CB
:1032700081B402D0D88001D0D89006B003D002E249
:10328000069001D00680006A06B0002A01500016A0
:1032900007E010DC02019051010A02E1906BC1D1FC
:1032A0000400800E050A006E800E03010619005C02
:1032B00002E10551DC08D8B0B4D10051040A010E76
:1032C000D8A4000E016E0051050A010ED8A4000E0C
:1032D000006E01500012D8B4C7D0020E446F100E19
:1032E000456F9F0E466F020E476F080E486F06EC43
:1032F00007F0030E0B6E080E0C6E770E0D6E0D2E82
:10330000FED70C2EFCD70B2EFAD7020E0301446F0A
:10331000100E456F850E466F020E476F080E486F00
:1033200006EC07F00B0E0B6E260E0C6E5D0E0D6E8E
:103330000D2EFED70C2EFCD70B2EFAD70000000066
:103340000400020E0301446F100E456F3A0E466FE3
:10335000020E476F080E486F06EC07F0070E0B6E63
:10336000170E0C6E6A0E0D6E0D2EFED70C2EFCD7AE
:103370000B2EFAD70000020E0301446F100E456FAA
:10338000310E466F020E476F080E486F06EC07F0CD
:103390000B0E0B6E260E0C6E5D0E0D6E0D2EFED7F7
:1033A0000C2EFCD70B2EFAD7000000000400020EF2
:1033B0000301446F100E456F430E466F020E476FB8
:1033C000080E486F06EC07F0070E0B6E170E0C6E1A
:1033D0006A0E0D6E0D2EFED70C2EFCD70B2EFAD7D3
:1033E0000000020E0301446F100E456F550E466F2C
:1033F000020E476F080E486F06EC07F00B0E0B6EBF
:10340000260E0C6E5D0E0D6E0D2EFED70C2EFCD70B
:103410000B2EFAD7000000000400020E0301446FD7
:10342000100E456F4C0E466F020E476F080E486F28
:1034300006EC07F0030E0B6E080E0C6E770E0D6E89
:103440000D2EFED70C2EFCD70B2EFAD7020E030141
:10345000446F100E456F0D0E466F020E476F080E3B
:10346000486F06EC07F0C3D003010051000AD8B43E
:10347000BED0010E446F456B040E466F020E476FBF
:10348000080E486F06EC07F0030E0B6E080E0C6E6C
:10349000770E0D6E0D2EFED70C2EFCD70B2EFAD705
:1034A000010E0301446F456B160E466F020E476F07
:1034B000080E486F06EC07F00B0E0B6E260E0C6E16
:1034C0005D0E0D6E0D2EFED70C2EFCD70B2EFAD7EF
:1034D000000000000400010E0301446F456B280E3C
:1034E000466F020E476F080E486F06EC07F0070E96
:1034F0000B6E170E0C6E6A0E0D6E0D2EFED70C2E77
:10350000FCD70B2EFAD70000010E0301446F456B68
:103510001F0E466F020E476F080E486F06EC07F04D
:103520000B0E0B6E260E0C6E5D0E0D6E0D2EFED765
:103530000C2EFCD70B2EFAD7000000000400010E61
:103540000301446F456B6A0E466F020E476F080E0B
:10355000486F06EC07F0070E0B6E170E0C6E6A0E26
:103560000D6E0D2EFED70C2EFCD70B2EFAD70000B9
:10357000010E0301446F456B610E466F020E476FEB
:10358000080E486F06EC07F00B0E0B6E260E0C6E45
:103590005D0E0D6E0D2EFED70C2EFCD70B2EFAD71E
:1035A000000000000400010E0301446F456B730E20
:1035B000466F020E476F080E486F06EC07F0030EC9
:1035C0000B6E080E0C6E770E0D6E0D2EFED70C2EA8
:1035D000FCD70B2EFAD7010E0301446F456B7C0E0E
:1035E000466F020E476F080E486F06EC07F00B0E91
:1035F0000B6E260E0C6E5D0E0D6E0D2EFED70C2E74
:10360000FCD70B2EFAD7000000000400100E0201B8
:103610008E6F270E8F6FAAC229F3ABC22AF384ECF8
:1036200015F0120021C300F00032009E0032009E0F
:103630000032009E0032009E0A0E0002F3CF01F01D
:103640000F0E03012115006E01500026120045ECFB
:1036500000F0DEC25DF30EEC00F003015D6B0EECDA
:1036600000F0AE0E03015D6F0EEC00F00201E651BA
:10367000020A010ED8A4000E016EE651030A010EE3
:10368000D8A4000E006E01500012D8B497D0D50E09
:1036900003015D6F0EEC00F0800E03015D6F0EEC18
:1036A00000F0A80E03015D6F0EEC00F03F0E030169
:1036B0005D6F0EEC00F0D30E03015D6F0EEC00F0B9
:1036C0000201E651020A05E1DFC25DF30EEC00F0F3
:1036D00007D00201DF511F0F03015D6F0EEC00F0F8
:1036E000400E03015D6F0EEC00F08D0E03015D6F67
:1036F0000EEC00F0140E03015D6F0EEC00F0810E75
:1037000003015D6F0EEC00F0B40E03015D6F0EEC73
:1037100000F0D90E03015D6F0EEC00F0220E0301E4
:103720005D6F0EEC00F0200E03015D6F0EEC00F0FB
:10373000020E03015D6F0EEC00F0210E03015D6FC0
:103740000EEC00F003015D6B0EEC00F07F0E030148
:103750005D6F0EEC00F02E0E03015D6F0EEC00F0BD
:103760000201E651020A0BE1A00E03015D6F0EECAF
:1037700000F0C00E03015D6F0EEC00F00AD0A10E48
:1037800003015D6F0EEC00F0C80E03015D6F0EECDF
:1037900000F0DA0E03015D6F0EEC00F0020E030183
:1037A0005D6F0EEC00F0DB0E03015D6F0EEC00F0C0
:1037B000400E03015D6F0EEC00F08AD0D50E0301C0
:1037C0005D6F0EEC00F0800E03015D6F0EEC00F0FB
:1037D000A80E03015D6F0EEC00F03F0E03015D6F5C
:1037E0000EEC00F0D30E03015D6F0EEC00F0DFC2B3
:1037F0005DF30EEC00F0400E03015D6F0EEC00F087
:103800008D0E03015D6F0EEC00F0140E03015D6F71
:103810000EEC00F0810E03015D6F0EEC00F0FF0E68
:1038200003015D6F0EEC00F0D90E03015D6F0EEC2D
:1038300000F0F10E03015D6F0EEC00F0200E0301AD
:103840005D6F0EEC00F0020E03015D6F0EEC00F0F8
:10385000210E03015D6F0EEC00F003015D6B0EECB9
:1038600000F07F0E03015D6F0EEC00F02E0E0301E1
:103870005D6F0EEC00F00201E651040A0BE1A00EB0
:1038800003015D6F0EEC00F0C00E03015D6F0EECE6
:1038900000F00AD0A10E03015D6F0EEC00F0C80E1F
:1038A00003015D6F0EEC00F0DA0E03015D6F0EECAC
:1038B00000F0120E03015D6F0EEC00F0DB0E030151
:1038C0005D6F0EEC00F0400E03015D6F0EEC00F03A
:1038D000A40E03015D6F0EEC00F0A60E03015D6FF8
:1038E0000EEC00F0C4EC00F0030E0B6E080E0C6E34
:1038F000770E0D6E0D2EFED70C2EFCD70B2EFAD7A1
:1039000045EC00F0DEC25DF30EEC00F0400E03016A
:103910005D6F0EEC00F00201E651020A010ED8A420
:10392000000E016EE651030A010ED8A4000E006ECF
:103930000150001219E00301226B2251030813E326
:1039400022C358F3596B81EC00F00301216B030192
:10395000800E215D05E2212B5D6B0EEC00F0F7D7A8
:103960000301222BEAD718D00301226B225107084A
:1039700013E322C358F3596B81EC00F00301216B70
:103980000301800E215D05E2212B5D6B0EEC00F042
:10399000F7D70301222BEAD7C4EC00F0AF0E0301E6
:1039A000236F79EC17F01200A69C21C3A9FFA69EF5
:1039B000A680A8CF00F01200DA0E0201E16F0C0E13
:1039C000E26F440EE36F030EE46FC26A0101891DCA
:1039D000006E0050C116070EC012C08EC2801200C9
:1039E00004008B908B9C8B9E03010051000A02E126
:1039F0008A8C8A8E0051040A010ED8A4000E016E32
:103A00000051050A010ED8A4000E006E01500012EC
:103A100019E0446B400E456FCC0E466F010E476FA8
:103A2000040E486F06EC07F0020E0301446F400ECF
:103A3000456FC70E466F010E476F040E486F06ECC8
:103A400007F01CD003010051000A18E0446B040E7B
:103A5000456FE00E466F010E476F040E486F06EC8F
:103A600007F0010E0301446F040E456FDB0E466F35
:103A7000010E476F040E486F06EC07F011EC16F0CC
:103A8000FF0E0301426F5FC243F342EC0EF0FE0EE5
:103A90000301426FDBC243F342EC0EF0FD0E030163
:103AA000426FDAC243F342EC0EF003010051000A08
:103AB00018E1800E006E800E0819005C02E10751CB
:103AC000960802E38A9C0DD0800E006E800E0819C5
:103AD000005C02E10751FA0803E3819C819E01D05A
:103AE000819E800E006E800E0819005C02E1075175
:103AF000960802E38B800CD0800E006E800E0819B1
:103B0000005C02E10751FA0802E38B8C01D08B8E36
:103B100002018E6B8F6B100EA86F270EA96F8BECB6
:103B200017F007C39BF208C39CF27CEC0BF0899E54
:103B3000898604001200040003010051040A010EEA
:103B4000D8A4000E016E0051050A010ED8A4000E83
:103B5000006E0150001248E0446B100E456FD20E0B
:103B6000466F010E476F080E486F06EC07F0020E15
:103B70000301446F100E456F8A0E466F010E476FAA
:103B8000080E486F06EC07F0040E0301446F100E98
:103B9000456F660E466F010E476F080E486F06ECC4
:103BA00007F0060E0301446F100E456F5D0E466F61
:103BB000010E476F080E486F06EC07F00201AC5388
:103BC000010ED8A4000E006E9D5100160CE00301FA
:103BD000446B700E456F5B0E466F010E476F010E12
:103BE000486F06EC07F065D003010051000A61E060
:103BF000446B456B800E466F010E476F080E486F91
:103C000006EC07F0010E0301446F456B770E466F1B
:103C1000010E476F080E486F06EC07F003010051D4
:103C2000010A19E1446B090E456F6F0E466F010ED4
:103C3000476F070E486F06EC07F0010E0301446F53
:103C4000090E456F510E466F010E476F070E486F04
:103C500006EC07F019D00301446B090E456F480EBE
:103C6000466F010E476F080E486F06EC07F0010E15
:103C70000301446F090E456F3F0E466F010E476FFB
:103C8000080E486F06EC07F00201AC53010ED8A4F1
:103C9000000E006E9D5100160CE00301446B080EEF
:103CA000456F590E466F010E476F010E486F06ECC7
:103CB00007F004000201DC6BD96B7CEC0BF0120006
:103CC0000900F5CFE6FF0006FBE10106F9E112006D
:103CD0000400010E0301216F67DE00C000F3020E35
:103CE000216F62DE0050010A03E1010E02019D6FA7
:103CF000030E0301216F58DE00C021F393DC00C0E6
:103D000001F3000E026F040E216F4EDE00C021F39E
:103D100089DC0A0E0002F3CFFEF2F4CFFFF2050EAB
:103D2000216F42DE00C021F37DDC0A0E0002F3CFDA
:103D3000EEF2F4CFEFF2060E216F36DE00C021F373
:103D400071DC0A0E0002F3CFECF2F4CFEDF2090EB3
:103D5000216F2ADE00C021F365DC0A0E0002F3CFDA
:103D6000EAF2F4CFEBF20400100E216F1DDE00C06A
:103D700021F358DC640E0002F3CF1FF3F4CF20F3DD
:103D8000110E216F11DE00C021F34CDC00501F2505
:103D90000D6F000E20210E6F120E216F05DE00C088
:103DA00021F340DC640E0002F3CF1FF3F4CF20F3C5
:103DB000130E216FF9DD00C021F334DC00501F2504
:103DC0000B6F000E20210C6F140E216FEDDD00C073
:103DD00021F328DC640E0002F3CF1FF3F4CF20F3AD
:103DE000150E216FE1DD00C021F31CDC00501F2502
:103DF000116F000E2021126F160E216FD5DD00C04D
:103E000021F310DC640E0002F3CF1FF3F4CF20F394
:103E1000170E216FC9DD00C021F304DC00501F25FF
:103E20000F6F000E2021106F180E216FBDDD00C036
:103E300021F312EC1BF0640E0002F3CF1FF3F4CF5A
:103E400020F3190E216FB0DD00C021F312EC1BF03E
:103E500000501F25096F000E20210A6F200E216FD0
:103E6000A3DD00C021F312EC1BF0640E0002F3CFBF
:103E70001FF3F4CF20F3210E216F96DD00C021F354
:103E800012EC1BF000501F25176F000E2021186F39
:103E9000220E216F89DD00C021F312EC1BF0640EAD
:103EA0000002F3CF1FF3F4CF20F3230E216F7CDD4C
:103EB00000C021F312EC1BF000501F251B6F000EF9
:103EC00020211C6F240E216F6FDD00C021F312EC46
:103ED0001BF0640E0002F3CF1FF3F4CF20F3250E86
:103EE000216F62DD00C021F312EC1BF000501F2592
:103EF000196F000E20211A6F260E216F55DD00C0AC
:103F000021F312EC1BF0640E0002F3CF1FF3F4CF89
:103F100020F3270E216F48DD00C021F312EC1BF0C7
:103F200000501F25156F000E2021166F280E216FDF
:103F30003BDD00C021F312EC1BF0640E0002F3CF56
:103F40001FF3F4CF20F3290E216F2EDD00C021F3E3
:103F500012EC1BF000501F25136F000E2021146F70
:103F600004001200070EB46E600ED36E9B8C806A44
:103F7000816A826A896A8A6A8B6A030E926EF90E76
:103F8000936E946A19DD0D0EC16EF19EF29E1200C1
:103F900003010051040A010ED8A4000E016E005165
:103FA000050A010ED8A4000E006E015000120CE0AC
:103FB000446B0A0E456F350E466F010E476F090EB2
:103FC000486F06EC07F00FD003010051000A0BE028
:103FD000446B030E456FB80E466F010E476F090E16
:103FE000486F06EC07F004000B0E0B6E260E0C6EED
:103FF0005D0E0D6E0D2EFED70C2EFCD70B2EFAD7B4
:104000000000000004000B0E0B6E260E0C6E5D0E01
:104010000D6E0D2EFED70C2EFCD70B2EFAD70000FE
:10402000000004000B0E0B6E260E0C6E5D0E0D6E66
:104030000D2EFED70C2EFCD70B2EFAD70000000059
:1040400004000B0E0B6E260E0C6E5D0E0D6E0D2E0B
:10405000FED70C2EFCD70B2EFAD700000000040070
:1040600003010051040A010ED8A4000E016E005194
:10407000050A010ED8A4000E006E015000120CE0DB
:10408000446B0A0E456FAE0E466F010E476F090E68
:10409000486F06EC07F00FD003010051000A0BE057
:1040A000446B030E456FA40E466F010E476F090E59
:1040B000486F06EC07F06BEC0BF0FF0E426F436BA2
:1040C00042EC0EF0FE0E0301426F436B42EC0EF029
:1040D000FD0E0301426F436B42EC0EF0010E020134
:1040E000DA6F010E0301296F2CEC14F00051040A61
:1040F000010ED8A4000E016E0051050A010ED8A4CD
:10410000000E006E015000120CE0446B700E456F03
:10411000C50E466F010E476F010E486F06EC07F0A3
:104120000FD003010051000A0BE0446B080E456FED
:10413000C30E466F010E476F010E486F06EC07F085
:10414000FADC1200810E0301366F0F0E376F386BE9
:10415000320E396F3A6B79EC11F002019E51001268
:104160003FE0898E8996060E0B6E130E0C6EAD0E17
:104170000D6E0D2EFED70C2EFCD70B2EFAD700009D
:10418000000004009E51000A010ED8A4000E016E2A
:1041900081B002D0D89001D0D880006AD8B0002A6F
:1041A0000150001605E0B1EC11F00001F76B16D0DC
:1041B00017DC0001F76B810E0301366F0F0E376FAE
:1041C000386B320E396F3A6B79EC11F0005204E023
:1041D0008BEC17F00400EFD702019E6B7CEC0BF028
:1041E000810E0301366F0F0E376F050E386F320EDA
:1041F000396F3A6B79EC11F000524FE00400000186
:10420000F751000A20E1010EF76F5FC2FBF1DBC23C
:10421000FAF1DAC2F9F102015F6BDB6B010EDA6FC2
:104220000301446B1DEC04F05FC244F37AEC08F028
:10423000DAC229F32CEC14F09DC2D1F102019D6B7E
:104240007CEC0BF018D00001F76BFBC15FF2FAC1F8
:10425000DBF2F9C1DAF2FBC144F37AEC08F0DBC21D
:1042600044F31DEC04F0DAC229F32CEC14F0D1C1B4
:104270009DF27CEC0BF0810E0301366F0F0E376F51
:10428000050E386F320E396F3A6B79EC11F000522F
:1042900004E08BEC17F00400EED7810E0301366FBB
:1042A0000F0E376F040E386F320E396F3A6B79ECA0
:1042B00011F00001F751000A010ED8A4000E016EA2
:1042C0000150001624E0040002019D51000A03E1A0
:1042D000010E9D6F01D09D6B020E0301426F9DC2C6
:1042E00043F342EC0EF07CEC0BF0810E0301366FD1
:1042F0000F0E376F040E386F320E396F3A6B79EC50
:1043000011F0005204E08BEC17F00400EED712001D
:10431000810E0301366F0F0E376F386B320E396F17
:104320003A6B79EC11F00052D8B493D0060E0B6EB4
:10433000130E0C6EAD0E0D6E0D2EFED70C2EFCD78F
:104340000B2EFAD700000000040081A00FD002015C
:10435000DA51000A03E1010EDA6F01D0DA6BDAC23A
:1043600029F32CEC14F07CEC0BF062D00101C2516B
:10437000010A02E1C26B02D0010EC26FC251010AF2
:104380002CE103010051040A010ED8A4000E016EB5
:104390000051050A010ED8A4000E006E0150001253
:1043A0000CE0446B700E456F970E466F010E476F21
:1043B000010E486F06EC07F00FD003010051000A10
:1043C0000BE0446B080E456F950E466F010E476F6C
:1043D000010E486F06EC07F02BD003010051040AD0
:1043E000010ED8A4000E016E0051050A010ED8A4DA
:1043F000000E006E015000120CE0446B700E456F11
:10440000930E466F010E476F010E486F06EC07F0E2
:104410000FD003010051000A0BE0446B080E456FFA
:10442000A20E466F010E476F010E486F06EC07F0B3
:10443000810E0301366F0F0E376F386B320E396FF6
:104440003A6B79EC11F0005204E08BEC17F00400A9
:10445000EFD7810E0301366F0F0E376F050E386FE1
:10446000320E396F3A6B79EC11F000523CE00400E7
:104470000301810E366F0F0E376F050E386F320E47
:10448000396F3A6B79EC11F000522DE01F0E0201EA
:10449000DB5D010ED8B0000E006E0101C2510016A6
:1044A00007E00201DB2BDBC244F31DEC04F015D066
:1044B0000101C253010ED8A4000E016E1F0E0201AD
:1044C0005F5D010ED8B0000E006E0150001605E0D1
:1044D0005F2B5FC244F37AEC08F07CEC0BF08BECC2
:1044E00017F00400C5D7810E0301366F0F0E376F2A
:1044F000040E386F320E396F3A6B79EC11F000010F
:10450000F751000A010ED8A4000E016E01500016EA
:104510003CE00400810E0301366F0F0E376F040E6E
:10452000386F320E396F3A6B79EC11F000522DE092
:104530000201DB510008010ED8B0000E006E01012F
:10454000C251001607E00201DB07DBC244F31DEC99
:1045500004F015D00101C253010ED8A4000E016E63
:1045600002015F510008010ED8B0000E006E01502C
:10457000001605E05F075FC244F37AEC08F07CECBC
:104580000BF08BEC17F00400C5D712000301216B70
:10459000D4EC1CF000C0DEF20050000A05E1939C50
:1045A000939E8A8C8A8E04D0938C938E8A9C8A9E4A
:1045B0001200010E0301216FD4EC1CF000C0E6F2E2
:1045C000070E216FD4EC1CF000C0DFF2080E216F43
:1045D000D4EC1CF000C0E5F20201E651010A03E050
:1045E00027EC1BF060D0010EE76FE06B030E0301B8
:1045F0004E6FA7EC03F01A0E0C6EF80E0D6E0D2E1A
:10460000FED70C2EFCD70000030E03014E6FA7EC63
:1046100003F0060E0C6E300E0D6E0D2EFED70C2E16
:10462000FCD70000030E03014E6FA7EC03F0020E4F
:1046300003014E6FA7EC03F0020E03014E6FA7ECCF
:1046400003F0080E03014E6FA7EC03F003014E6B5D
:10465000A7EC03F0080E03014E6FA7EC03F0030173
:104660004E6BA7EC03F0010E03014E6FA7EC03F0B5
:104670001A0E0C6EF80E0D6E0D2EFED70C2EFCD7FA
:10468000000003014E6BA7EC03F0060E03014E6F12
:10469000A7EC03F003014E6BA7EC03F00C0E030133
:1046A0004E6FA7EC03F01200040003010051040A4E
:1046B000010ED8A4000E016E0051050A010ED8A407
:1046C000000E006E01500012D8B40AD1446B160ED1
:1046D000456FE90E466F000E476F070E486F06ECF8
:1046E00007F0020E0301446F040E456F590E466F2A
:1046F000000E476F0A0E486F06EC07F0040E030128
:10470000446F100E456F510E466F000E476F080E36
:10471000486F06EC07F0060E0C6E300E0D6E0D2E77
:10472000FED70C2EFCD70000040E0301446F100EC0
:10473000456F510E466F000E476F080E486F06EC2E
:1047400007F0060E0C6E300E0D6E0D2EFED70C2EE1
:10475000FCD70000040E0301446F100E456F510E8C
:10476000466F000E476F080E486F06EC07F0060E06
:104770000C6E300E0D6E0D2EFED70C2EFCD70000E9
:10478000060E0301446F040E456F460E466F000E81
:10479000476F0A0E486F06EC07F004000D0E0B6E13
:1047A0002D0E0C6ED70E0D6E0D2EFED70C2EFCD7D7
:1047B0000B2EFAD70000000004000B0E0B6E260E25
:1047C0000C6E5D0E0D6E0D2EFED70C2EFCD70B2E33
:1047D000FAD70000000004000301446B100E456F7F
:1047E000780E466F000E476F080E486F06EC07F014
:1047F000020E0301446F040E456F6D0E466F000EEE
:10480000476F0A0E486F06EC07F0040E0301446F71
:10481000100E456F640E466F000E476F080E486F0E
:1048200006EC07F0060E0301446F040E456F270ED9
:10483000466F000E476F0A0E486F06EC07F0040E35
:104840000B6E0C0E0C6E330E0D6E0D2EFED70C2E55
:10485000FCD70B2EFAD7000000000301446B100EAA
:10486000456F1E0E466F000E476F080E486F06EC30
:1048700007F0020E0301446F100E456F150E466FD0
:10488000000E476F080E486F06EC07F0040E030198
:10489000446F100E456F3D0E466F000E476F080EB9
:1048A000486F06EC07F0060E0301446F100E456FCB
:1048B000340E466F000E476F080E486F06EC07F087
:1048C00002019D530CE00301446B700E456F320EE4
:1048D000466F000E476F010E486F06EC07F028D1B7
:1048E00003010051000AD8B423D1446B040E456F74
:1048F000C40E466F000E476F070E486F06EC07F0B8
:10490000010E0301446F030E456FB90E466F000E92
:10491000476F0A0E486F06EC07F004000F0E0B6E8F
:10492000350E0C6E510E0D6E0D2EFED70C2EFCD7D3
:104930000B2EFAD704000B0E0B6E260E0C6E5D0EBE
:104940000D6E0D2EFED70C2EFCD70B2EFAD70000C5
:10495000000004000301446B040E456F510E466FC6
:10496000000E476F080E486F06EC07F0060E0C6E3F
:10497000300E0D6E0D2EFED70C2EFCD7000003015D
:10498000446B040E456F510E466F000E476F080EC4
:10499000486F06EC07F0060E0C6E300E0D6E0D2EF5
:1049A000FED70C2EFCD700000301446B040E456FAC
:1049B000510E466F000E476F080E486F06EC07F069
:1049C000060E0C6E300E0D6E0D2EFED70C2EFCD783
:1049D0000000010E0301446F030E456FAE0E466FDB
:1049E000000E476F0A0E486F06EC07F004000D0E2C
:1049F0000B6E2D0E0C6ED70E0D6E0D2EFED70C2EDF
:104A0000FCD70B2EFAD70000000004000B0E0B6E33
:104A1000260E0C6E5D0E0D6E0D2EFED70C2EFCD7E5
:104A20000B2EFAD70000000004000301446B040EB3
:104A3000456FE00E466F000E476F080E486F06EC9C
:104A400007F0010E0301446F030E456FD50E466F4C
:104A5000000E476F0A0E486F06EC07F0040E0B6E4F
:104A60000C0E0C6E330E0D6E0D2EFED70C2EFCD7D9
:104A70000B2EFAD7000000000301446B456BCC0EEF
:104A8000466F000E476F080E486F06EC07F0010EE8
:104A90000301446F456B910E466F000E476F080E81
:104AA000486F06EC07F003010051010A19E1446B5D
:104AB000090E456F890E466F000E476F070E486F4F
:104AC00006EC07F0010E0301446F090E456F810EDD
:104AD000466F000E476F070E486F06EC07F019D0BF
:104AE0000301446B090E456FA50E466F000E476F1C
:104AF000080E486F06EC07F0010E0301446F090E23
:104B0000456F9C0E466F000E476F080E486F06EC0F
:104B100007F002019D530CE00301446B080E456F42
:104B20009A0E466F000E476F010E486F06EC07F0B5
:104B30000400120013EC29F0D0B603D0010E0101DD
:104B4000A16F01018986550E9925516E2D0EA02564
:104B5000586EB2EC1FF0720E9A25526E320E9F25DF
:104B6000576E030E0B6E080E0C6E770E0D6E0D2E2B
:104B7000FED70C2EFCD70B2EFAD704001E0E9B2559
:104B8000536E3B0E9E25566E68EC1EF0FFDC420E07
:104B900001019C25546E050E0B6E0F0E0C6EF10E6E
:104BA0000D6E0D2EFED70C2EFCD70B2EFAD704005F
:104BB00081B802D0028001D0029081BA02D0D880A0
:104BC00001D0D89002A003D002E3028001D002906D
:104BD00002A003D0010E0201AC6FEBDC81B802D061
:104BE000028001D0029081BA02D0D88001D0D89042
:104BF00002A003D002E3028001D0029081B002D073
:104C0000D88001D0D89002A003D002E3028001D066
:104C1000029002A03CD0030100510A0A0CE1446B4F
:104C2000030E456FEF0E466F010E476F090E486F7A
:104C300006EC07F00FD003010051000A0BE0446BB3
:104C40000C0E456FE50E466F010E476F090E486F5B
:104C500006EC07F0FF0E0301446F7AEC08F0FF0E3C
:104C6000446F1DEC04F0010E296F2CEC14F00B0EB8
:104C70000B6E260E0C6E5D0E0D6E0D2EFED70C2EDD
:104C8000FCD70B2EFAD7000000000400F0D71C0E52
:104C900001019D25556E0400A151000A010ED8A402
:104CA000000E016E0201AC51000A010ED8A4000EE4
:104CB000006E015000161DE06BEC0BF0FF0E426F12
:104CC000436B42EC0EF0FE0E0301426F436B42EC6D
:104CD0000EF0FD0E0301426F436B42EC0EF0010E2D
:104CE0000201DA6F010E0301296F2CEC14F0DCDCF9
:104CF00035D00101A151010A010ED8A4000E016EA8
:104D00000201AC51000A010ED8A4000E006E015041
:104D1000001622E0FF0E0301216FD4EC1CF000C04E
:104D20005FF2FE0E216FD4EC1CF000C0DBF2FD0E32
:104D3000216FD4EC1CF000C0DAF2DBC244F31DECAE
:104D400004F05FC244F37AEC08F0DAC229F32CECE9
:104D500014F09BEC1DF002D0C8EC1FF07CEC0BF0C3
:104D600004008BEC17F00201AC51000A03E1A2EC45
:104D700020F002D088EC21F0F3D7FFD75357523DF3
:104D8000302E3030005057523D302E30570020200A
:104D90002020202020202020002E00433D20202005
:104DA000307046004C3D302E30307548004657205C
:104DB00076657220322E35000C100E0D120B10137A
:104DC0006D696E6920626F6172640020202020206E
:104DD0002020200020202020202020202020002013
:104DE0002020202020202000433D2020307046003D
:104DF0004C3D302E307548005357523D302E3030E8
:104E0000002E00433D202020307046004C3D302EC7
:104E1000303075480046572076657220322E3500B6
:104E20006D696E6920626F617264004154552D3165
:104E30003030005057523D302E3057002020202077
:104E400020202020202000202020202020202000A2
:104E50004154552D3130300020005F002E00005F9E
:104E6000002E0020005057523D302E30570053572F
:104E7000523D302E30300052455345542020200002
:104E80005057523D302E3057005357523D302E3040
:104E900030005245534554202020000054455354BF
:104EA000204D4F444500433D202020307046004CAB
:104EB0003D302E3031754800433D20203070460093
:104EC0002E002E00433D202020307046004C3D3007
:104ED0002E30307548004C3D302E30754800535709
:104EE000523D302E3030005057523D302E3057005A
:104EF000305357523D302E30300063006C006C0050
:104F00000D07020C1B091216006300202020202030
:104F1000202020200020202020202020202000549D
:104F2000455354204D4F444500016C006C005455CE
:104F30004E45005741495400005057523D302E30E5
:104F4000570054554E45005741495400464153546B
:104F50002054455354004641535420544553540063
:104F6000000000433D20202070460020202020200B
:104F7000202020005357523D20202020004F56452E
:104F8000524C4F4144004F5645524C4F4144002033
:104F900020202020202020004F5645524C4F4144D5
:104FA0000020202020202020200020202020202041
:104FB0002020002020202020202020004F56455275
:104FC0004C4F4144000000004F5645524C4F414465
:104FD0000020202020202020200020202020202011
:104FE0002020005357523D20202020004F5645528C
:104FF0004C4F414400102700302E303000302E300E
:105000003000000000002020202020202020001060
:10501000270000004C3D202020207548004C3D20FA
:1050200020207548004C3D20202020754800433D3D
:1050300020202020704600433D2020202070460084
:10504000FD0000FD01000000000000005F00000006
:1050500007000700147F147F14242A7F2A122313C9
:1050600008646236495522500005030000001C22E6
:1050700041000041221C00082A1C2A0808083E089A
:105080000800503000000808080808003030000010
:1050900020100804023E5149453E00427F40004234
:1050A000615149462141454B311814127F10274563
:1050B0004545393C4A49493001710905033649499A
:1050C0004936064949291E0036360000005636008A
:1050D000000008142241141414141441221408006E
:1050E0000201510906324979413E7E1111117E7F3C
:1050F000494949363E414141227F4141221C7F4975
:105100004949417F090901013E414151327F080867
:10511000087F00417F41002040413F017F08142269
:10512000417F404040407F0204027F7F0408107F9F
:105130003E4141413E7F090909063E4151215E7FC2
:1051400009192946464949493101017F01013F407A
:1051500040403F1F2040201F7F2018207F631408FD
:1051600014630304780403615149454300007F41FF
:1051700041020408102041417F00000402010204A2
:105180004040404040000102040020545454787FC5
:10519000484444383844444420384444487F3854D0
:1051A000545418087E090102081454543C7F080422
:1051B000047800447D40002040443D00007F1028DA
:1051C0004400417F40007C041804787C0804047883
:1051D00038444444387C14141408081414187C7C93
:1051E000080404084854545420043F4440203C40E0
:1051F00040207C1C2040201C3C4030403C44281077
:1052000028440C5050503C4464544C4400083641EF
:105210000000007F0000004136080008082A1C0832
:10522000081C2A0808FF10EE15F0C90E006E030EC8
:10523000016E7C0EF66E4D0EF76E000EF86E60EC91
:105240001EF01200FFFFFFFFFFFFFFFFFFFFFFFF4A
:020000040030CA
:0D000100081A11FF8181FF0FC00FE00F40B2
:0200000400F00A
:100000004E010015130500010200FFFFFFFFFFFF77
:1000100001100220045010002200FFFFFFFFFFFF2D
:1000200000100022004701000220FFFFFFFFFFFF3A
:10003000FFFFFFFFFFFFFFFFFFFFFFFFFFFFFFFFD0
:10004000FFFFFFFFFFFFFFFFFFFFFFFFFFFFFFFFC0
:10005000FFFFFFFFFFFFFFFFFFFFFFFFFFFFFFFFB0
:10006000FFFFFFFFFFFFFFFFFFFFFFFFFFFFFFFFA0
:10007000FFFFFFFFFFFFFFFFFFFFFFFFFFFFFFFF90
:10008000FFFFFFFFFFFFFFFFFFFFFFFFFFFFFFFF80
:10009000FFFFFFFFFFFFFFFFFFFFFFFFFFFFFFFF70
:1000A000FFFFFFFFFFFFFFFFFFFFFFFFFFFFFFFF60
:1000B000FFFFFFFFFFFFFFFFFFFFFFFFFFFFFFFF50
:1000C000FFFFFFFFFFFFFFFFFFFFFFFFFFFFFFFF40
:1000D000FFFFFFFFFFFFFFFFFFFFFFFFFFFFFFFF30
:1000E000FFFFFFFFFFFFFFFFFFFFFFFFFFFFFFFF20
:1000F000FFFFFFFFFFFFFFFFFFFFFFFFFFFFFFFF10
:00000001FF
